:1000000000308A00192800002230840000080319FB
:1000100018280130F800F701F70B0C28F80B0B2813
:100020004A30F700F70B122800000000800B092867
:10003000003484011F30830583161F129F121B0892
:1000400080399B0007309C001F129F121B088039CB
:100050009B0083121F109412831606118614061239
:10006000003083129400831694000108C7390838C1
:100070008100831290010030F80092000030831656
:10008000920007309C0005080330F700F70B462864
:100090001C0883120D1383169D018F010F08061093
:1000A000831206140430A100AF30A2000420A10B7B
:1000B000542883160610831206103230A200042042
:0600C00083164F286300C7
:04400E00093FFC3F2B
:00000001FF
